:100305007D577C027F101203687D017F0112043B3B
:100315007D017F0812043BE4FD7F011204467D0147
:100325007F081204467D2C7C01E4FF1201F57D0F48
:100335007F0F12045C7F01120451E4FD7F0102036B
:01034500B403
:10039D007B027D017F021202587D017F021204094A
:0703AD00120305D2AF80FE30
:0300030002046E86
:01046E00325B
:03000B0002046F7D
:01046F00325A
:0300130002047074
:010470003259
:03001B000204716B
:010471003258
:0300230002047262
:010472003257
:03002B0002047359
:010473003256
:0300330002047450
:010474003255
:03003B0002047547
:010475003254
:030043000202B7FF
:1002B700C0E0C0F0C083C082C0D075D000C000C00D
:1002C70001C002C003C004C005C006C0077D017F8E
:1002D700021203E0EF7D017F0260051203CA80036B
:1002E700120409D007D006D005D004D003D002D01D
:0E02F70001D000D0D0D082D083D0F0D0E03241
:03004B0002047636
:010476003253
:030053000204772D
:010477003252
:10034600E4F5D1F5D2F5D3F5D4F5D5F5D6F5D7F54F
:10035600DAF5DBF5DCF5DDF5DEF5DF53A9FD53B99E
:02036600FD2276
:10036800ED5403FEE5D254CC4F4EF5D2AE04ED78F1
:0B03780002CEC313CE13D8F9F5D32238
:0B043B00EFBD010342DA22F452DA2286
:0B044600EFBD010342D122F452D1228D
:1001000053DA7FEF24FE603E24FE605824FC6071C9
:1001100024F870030201A024F070030201BA24E065
:1001200070030201D8243F60030201F4ED5403FF81
:10013000E5D454FC4FF5D4AE04ED7802CEC313CE13
:1001400013D8F9F5D522ED540325E025E0FFE5D4D9
:1001500054F34FF5D4AE04ED7802CEC313CE13D8CA
:10016000F9F5D622ED5403C454F0FFE5D454CF4F33
:10017000F5D4AE04ED7802CEC313CE13D8F9F5D77B
:1001800022ED5403C4333354C0FFE5D4543F4FF53C
:10019000D4AE04ED7802CEC313CE13D8F9F5DC2229
:1001A000ED5403FFE5DB54FC4FF5DBAE04ED7802C4
:1001B000CEC313CE13D8F9F5DD22ED540325E02587
:1001C000E0FFE5DB54F34FF5DBAE04ED7802CEC380
:1001D00013CE13D8F9F5DE22ED5403C454F0FFE535
:1001E000DB54CF4FF5DBAE04ED7802CEC313CE1354
:0501F000D8F9F5DF2243
:1001F50043DA80EF14602114603C24027054ED54FE
:1002050003FFE5D454FC4FF5D4AE04ED7802CEC31C
:1002150013CE13D8F9F5D522ED540325E025E0FFDB
:10022500E5D454F34FF5D4AE04ED7802CEC313CE26
:1002350013D8F9F5D622ED5403C454F0FFE5D45490
:10024500CF4FF5D4AE04ED7802CEC313CE13D8F953
:03025500F5D722B8
:08045C00EDC454F04FF5DC2261
:0B045100EF600443D2802253D27F22D0
:1003B400EF600543A902800353A9FDED700443B91E
:0603C400022253B9FD22E4
:06046400E5D25440FF2226
:04046A0053D2BF2288
:1003F500E4F59AF591F5A1F59BF592F5A2F5A0F531
:0404050090F58022CC
:10025800EF701CEB7006EDF4529A529BBB0107ED50
:10026800F4529AED429BEB64027043ED429A22EFFE
:100278006401701CEB7006EDF452915292BB0107B9
:10028800EDF45291ED4292EB64027022ED4291221C
:10029800EF64027019EB7006EDF452A152A2BB0193
:0F02A80007EDF452A1ED42A2BB0203ED42A122E9
:10041C00EF70028D80BF01028D90BF02028DA02271
:10040900EF7003ED4280BF0103ED4290BF0203ED9F
:0304190042A022DC
:1003CA00EF7004EDF45280BF0104EDF45290BF02C5
:0603DA0004EDF452A02224
:0F042C00EF7003AF8022BF0103AF9022AFA02279
:1003E000EF7005E5805DFF22BF0105E5905DFF220E
:0503F000E5A05DFF2205
:0300000002038375
:1003830078FFE4F6D8FD9000007F007E01E4F0A33F
:0A039300DFFCDEFA75810702039D0E
:00000001FF
